:020000020000FC
:100000006FC16EC16DC10EC10DC10CC105C068C10B
:1000100067C166C165C164C1000062BE03951895E1
:10002000F894C4FD32C0C3FD70C0C2FD97C0C1FDCD
:10003000DFC0C5FD19C0C6FF17C0C260CE7FF894EF
:10004000B0E8B0937000B1E0B0937100B2E0B0934B
:100050007200B4E0B0937300B8E0B0937400B0E104
:10006000B09375007894DCC0F894BFEFB093700043
:10007000B0937100B0937200B0937300B0937400AA
:10008000B0937500C5987894CBC0C5FD1BC0BB2745
:10009000B09380008824B0938600C39AC09AD89AFF
:1000A000D99ADC9ADF9ACF7EC860BAEAB09376001C
:1000B000B8E21B2EB8E8A694A1FE6EC0B0E8AB2E45
:1000C000B8E86AC0B0918600BB2391F4BFEFB0934B
:1000D000860080928000C59AA7FCC398A6FCC098B1
:1000E000A5FCD898A4FCD998A3FCDC98A2FCDF98C6
:1000F000B0918000482D4B1B463030F0C39AC09A17
:10010000D89AD99ADC9ADF9A8BC0BB27B093860025
:100110008824112031F0C5FF83C0C77FC061BFEFC5
:100120003BC0C77FC598C260B0E8AB2EF894BB2730
:10013000B0937600B0E8B0937000B1E0B093710076
:10014000B2E0B0937200B4E0B0937300B8E0B09343
:100150007400B0E1B0937500789462C0C5FF01C02F
:1001600008C076FC03C0B4E03B2E5AC03320A9F18E
:1001700057C076FEF8CFA694F894BB27B0937000D2
:10018000B0937100B0937200B0937300B093740099
:10019000B09375007894BAEAA7FE03C0B0937000DC
:1001A0003FC0A6FE03C0B09371003AC0A5FE03C0D5
:1001B000B093720035C0A4FE03C0B093730030C08A
:1001C000A3FE03C0B09374002BC0A2FE03C0B09383
:1001D000750026C0B0E8AB2EDECFCB7FC860BAEA90
:1001E000B0937600B8E2C59A1B2EB8E8D5CF18C0F8
:1001F000C5FF16C0C460CD7FB4E03B2EBB27F8948A
:10020000B0937100B0937200B0937300B093740018
:10021000B0937500BAEAB09370007894B0E8AB2E52
:100220007C2E0895BEB5BB2369F0B0917600B0FF77
:1002300002C0C69A01C0C698B69508F4B068B093DB
:100240007600189578943A941A948394B09170003B
:10025000B7FF02C0BC9A01C0BC988894B69508F458
:10026000B068B0937000B0917100B7FF02C0BA9A45
:1002700001C0BA98B69508F4B068B0937100B09117
:100280007200B7FF02C0B99A01C0B998B69508F4D8
:10029000B068B0937200B0917300B7FF02C0D29AF9
:1002A00001C0D298B69508F4B068B0937300B091CD
:1002B0007400B7FF02C0D39A01C0D398B69508F472
:1002C000B068B0937400B0917500B7FF02C0D59AC2
:1002D00001C0D598B69508F4B068B093750018952C
:1002E0009FED9DBF15E02AE03FE09EE2AEEFB1E05A
:1002F0004B2EBB275B2EB2E76B2E62BEBD9AC59814
:10030000BE9AC6980027DD27EE27B6E6B9BFBBE048
:10031000BFBDBFEFBAEABDBDB5E5BCBDC1E07C2E37
:10032000BFEFB0937000B0937100B0937200B093C0
:100330007300B0937400B0937500C39AC09AD89AB2
:10034000D89AD99ADC9ADF9ABB9AB89AD09AD09A5E
:10035000D19AD49AD79ABB27B0938000B0938100EA
:10036000B0938200B0938300B0938400B093850073
:10037000B0938600B0938700B0938800B093890053
:10038000B0938A00B0938B00B0E8AB2EBCEFBB2ECD
:10039000B0937A008824F894002753BEC1E0C59832
:1003A000B0E8AB2EBB27B0937600BFEFB0937000E0
:1003B000B0937100B0937200B0937300B093740067
:1003C000B09375007894CE9BFECF62BE43BE789406
:1003D000CE9B04C0F894A017F0F2F9CFF89403175D
:1003E000D0F6021788F40117B8F4D5CF789418DE48
:1003F000CE9904C0F894A01770F2F8CFF8940917BA
:1004000050F262BE0027E3CFEE27D395D23070F3CF
:10041000C062CF7BDA95EACFDD27E395E23030F397
:08042000C064CF7DEA95E2CF34
:00000001FF
